:0A002600120DBF120F47120D6B22DE
:0300330002001AAE
:04001A0053D8EF3296
:100003008E138F14E5141514AE13700215134E607E
:0700130005120F3680EE22FA
:0300230002004692
:10004600C0E0C083C082C086758600C0D075D00867
:1000560030990E300807A20B929B853599C299D22A
:100066000F200F03020431C20F20020302025620A2
:100076000803020127E537C39550503E2009362074
:100086000633907F9BE030E303200E29300D12AF3C
:1000960037053774402FF582E4347EF583E01392FA
:1000A6000BAF37053774402FF582E4347EF583E0D5
:1000B600F53502042FC20802042F907FC7E4F0C270
:1000C60002300A0CC20A907FBB04F0C20802042F59
:1000D600907FC8E030E105C20802042F907FC9E096
:1000E600F550907DC0E013920A20092D20062A9033
:1000F6007F9BE030E303200E20300D11907DC1E0A0
:03004300020F00A9
:03000000020C618E
:4001060013920BA3E0F53575370302042F753702907DC1E0F53502042F753701C20802042FE537C3955050030201CF907FC6E030E107C210C20302042F907FC7E0F5509004
:400146007E40E013920A3009030201C720067220006F907F9BE030E303200E65300D10907E41E013929BA3E0F5997537038009907E41E0F599753702E537C39550401790B1
:400186007FC7E4F0C202200A0302042FC20A907FBB04F002042F300D12AF37053774402FF582E4347EF583E013920BAF37053774402FF582E4347EF583E0F535D20802045D
:4001C6002F753701C21002042F300903020251200679907F9BE030E303200E6F300D12AF37053774402FF582E4347EF583E013929BAF37053774402FF582E4347EF583E046
:40020600F599E537C395504017907FC7E4F0C202200A0302042FC20A907FBB04F002042F300D12AF37053774402FF582E4347EF583E013920BAF37053774402FF582E43483
:400246007EF583E0F535D20802042FC21002042F200803020308E537C39550503E200936200633907F9BE030E303200E29300D12AF37053774C02FF582E4347DF583E013DE
:40028600920BAF37053774C02FF582E4347DF583E0F53502042FC20802042F907FC9E4F0D202300A0CC20A907FBB04F0C20802042F907FC6E030E105C20802042F907FC765
:4002C600E0F550907E40E013920A20092D20062A907F9BE030E303200E20300D11907E41E013920BA3E0F53575370302042F753702907E41E0F53502042F753701C20802EF
:40030600042FE537C3955050030203B0907FC8E030E107C210C20302042F907FC9E0F550907DC0E013920A3009030203A820067220006F907F9BE030E303200E65300D1034
:40034600907DC1E013929BA3E0F5997537038009907DC1E0F599753702E537C395504017907FC9E4F0D202200A0302042FC20A907FBB04F002042F300D12AF37053774C0F5
:400386002FF582E4347DF583E013920BAF37053774C02FF582E4347DF583E0F535D20802042F753701C21002042F30090302042D200674907F9BE030E303200E6A300D128E
:4003C600AF37053774C02FF582E4347DF583E013929BAF37053774C02FF582E4347DF583E0F599E537C395504013907FC9E4F0D202300A35C20A907FBB04F0802C300D12CC
:40040600AF37053774C02FF582E4347DF583E013920BAF37053774C02FF582E4347DF583E0F535D2088002C210D21220980302056DC2982001030204DA201127AF360536F3
:4004460074802FF582E4347EF583E599F0300D4DAF36053674802FF582E4347EF583E598F0803A859910E510B54404D206802EE510B54304C2068025AF36053674802FF5AB
:4004860082E4347EF583E510F0300D11AF36053674802FF582E4347EF583E598F0D20CE536C39540500302056B907FB8E030E116E536C39440500302056B15361536052BDD
:4004C60043330102056B907FB7E536F0753600C20102056B201127AF36053674002FF582E4347EF583E599F0300D4DAF36053674002FF582E4347EF583E598F0803A859937
:4005060010E510B54404D206802EE510B54304C2068025AF36053674002FF582E4347EF583E510F0300D11AF36053674002FF582E4347EF583E598F0D20CE536C3954040CE
:4005460024907FB6E030E112E536C39440401615361536052B433301800B907FB9E536F0753600D201D212301205C212020056D0D0D086D082D083D0E032907FCAE030E1CA
:40058600030206ABE4F51374402513F582E4347DF583E0FFE5137C007B002438F9EC3400FAEF120D330513E513B418DBE538600C75C92075C8348539CA853ACBE53B1392BF
:4005C6000D929FE53C13920EE53D139211E53E6009907F98E054FBF08007907F98E04404F0E53F6009907F98E0547FF08007907F98E04480F0E545600BC209C206907F950E
:40060600E04402F0E546600CD206433301907F95E04402F0E547600DC2AFC208D200E4F550F537D2AFE5486005301102D206E5496015907F95E054FDF0907F9EE04402F0AA
:40064600907F98E054FDF0E54A600AD29CC298752C0175311EE54B6007C29CE4F536F52CE54C6003E4F536E54D6002D204E54E600AE54A7002F531E54E4233E54F601F9064
:400686007FD77411F07431F07412F07432F07413F07433F07414F07434F0D202D201D205E4907FCBF0A209E433FF652960058F29433301A206E433FF652A60058F2A4333BA
:4006C60001907F9BE05408B5250AE054086408F525433301907F9BE05410B5260AE054106410F526433301907F9BE05440B5270AE054406440F527433301907F9BE0542026
:40070600B5280AE054206420F528433301300435C2AF300118907FB8E020E127E5366009907FB7F0E4F536C201C2048016907FB6E020E10FE5366009907FB9F0E4F536D234
:4007460001C204D2AF20033730021B907FC6E020E12D907E40E013920A753701907FC7E0F550D2038019907FC8E020E112907DC0E013920A753701907FC9E0F550D20320E9
:400786001033200006E5376550702A30031A300209E4907FC7F0C2028007E4907FC9F0D202C203E4F550F537300A0AC20AC200907FBB7401F03010030208C5200303020805
:4007C600C5300E0A907F9BE030E3030208C53006030208C53009030208C5300262300D12AF37053774402FF582E4347EF583E0139219AF37053774402FF582E4347EF583CF
:40080600E0F514E537C39550502A300D12AF37053774402FF582E4347EF583E013920BAF37053774402FF582E4347EF583E0F535D208806BC208E4907FC7F0C20280603081
:400846000D12AF37053774C02FF582E4347DF583E0139219AF37053774C02FF582E4347DF583E0F514E537C39550502A300D12AF37053774C02FF582E4347DF583E013929F
:400886000BAF37053774C02FF582E4347DF583E0F535D2088009C208E4907FC9F0D202300D04A219929BD210C2AF85149920080D300A0AC20AC200907FBB7401F0D2AF9072
:4008C6007FBCE020E151E533604DE5317049E53330E108E4F52F753301800BA205E433F52FC205E4F533E4F5137E007B0074242513F9EE3400FA120CEDFF74002513F582D8
:40090600E4347DF583EFF00513E513B40CDB907FBD740CF075311022907FE9E0120D450A03000A77010AE30309410609F40809E80909D00A09DF0B00000B32907FEBE024EB
:40094600FE601614605724027076740F907FD4F07464907FD5F0020B39907FEAE070047F0280027F037582B575830FEFF07582AE75830FF07582A775830FF07582A07583BA
:400986000FF0907FEAE00475827B75830FF0740F907FD4F07476907FD5F0020B39907FEAE0FF120E48EA49600DEA907FD4F0E9907FD5F0020B39907FB4E04401F0020B39D4
:4009C600907FB4E04401F0020B39907F00E519F0907FB57401F0020B39907FEAE0F519020B39907FEAE0F518120D6B020B39907F00E518F0907FB57401F0020B39907FE822
:400A0600E0247F60241460312402705BA213E433FF25E0FFA217E4334F907F00F0E4A3F0907FB57402F0020B39E4907F00F0A3F0907FB57402F0020B39907FECE0F45480B6
:400A4600FFC4540FFFE054072F25E024B4F582E4347FF583E054FD907F00F0E4A3F0907FB57402F0020B39907FB4E04401F0020B39907FE8E024FE601D24026003020B3904
:400A8600907FEAE0B40105C213020B39907FB4E04401F0020B39907FEAE07038907FECE0F45480FFC4540FFFE054072F25E024B4F582E4347FF583E4F0907FECE05480FFCC
:400AC600131313541FFFE054072F907FD7F0E04420F0805F907FB4E04401F08056907FE8E024FE60182402704A907FEAE0B40104D213803F907FB4E04401F08036907FEA36
:400B0600E07020907FECE0F45480FFC4540FFFE054072F25E024B4F582E4347FF5837401F08010907FB4E04401F08007907FB4E04401F0907FB4E04402F022201503020B3E
:400B4600D3E53160021531E536604F65347045E532F460020532E532C39541403DC2AF300118907FB8E020E127907FB7E536F0C201E4F536F532F5348016907FB6E020E13D
:400B86000F907FB9E536F0D201E4F536F532F534D2AF8006853634E4F532E52C602F200C07907F9BE030E00FE52D6006E4F52D433301E4F5308014E530D39542500DE530DB
:400BC600B54206752D014333010530C20C22751201C214C218C213C217C215C212D216E4F518907F92E054FDF0907FAEE0FFD39213E433FEEF4EF0D2E843D820907FDE74DB
:400C060001F0907FDFF0907FAB74FFF0907FA9F0907FAAF05391EF907FAFE04401F0907FAEE0440DF0D2AFD2BCD219120EDAC214301503120580907FD8E065116008E0F5CA
:400C460011120B4180EA301407C21412091E80E03018DDC21812002680D622787FE4F6D8FD758150020CA8020BD4E493A3F8E493A34003F68001F208DFF48029E493A3F83B
:400C86005407240CC8C333C4540F4420C8834004F456800146F6DFE4800B0102040810204080900E04E47E019360BCA3FF543F30E509541FFEE493A360010ECF54C025E08E
:400CC60060A840B8E493A3FAE493A3F8E493A3C8C582C8CAC583CAF0A3C8C582C8CAC583CADFE9DEE780BEBB010689828A83E0225002E722BBFE02E32289828A83E4932242
:400D0600BB010CE58229F582E5833AF583E0225006E92582F8E622BBFE06E92582F8E222E58229F582E5833AF583E49322BB010689828A83F0225002F722BBFE01F322D0E1
:400D460083D082F8E4937012740193700DA3A393F8740193F5828883E4737402936860EFA3A3A380DFE4907F93F0907F9C7430F0907F967410F0907F947401F0907F9D04E2
:400D8600F0907F977420F0907F957403F0907F9E7484F0E4907F98F0907FC7F0907FC9F0907FCBF075984043A810907FDE741FF0907FDF740FF0D21522E4907F95F0907FF7
:400DC60094F0907F93F0907F9DE04402F0907F97E04402F0907F9DE054FDF0907F9C7420F0E4907F96F0907F9DE044FDF0E4907F97F0907F9E74FFF0E4907F98F0220C24D0
:400E0600000000000000000000000000013000013301013200013700015000013600013400C105C10CC103C10FC104C10EC111C10AC110C108C109C106C100C10DC181C109
:400E460082008F13E4F5147515FF75160F7517B9AB15AA16A917900001120D06B4031DAF140514EFB5130122120CED7E0029FFEE3AA9077515FFF516891780D47B007A006D
:400E8600790022C0E0C083C082C085C084C086758600907FC4E4F05391EF907FAB7404F0D086D084D085D082D083D0E032C0E0C083C082C085C084C086758600D2145391C7
:400EC600EF907FAB7401F0D086D084D085D082D083D0E032907FD6E054FBF0E04408F0301904E04402F07FF47E01120003907FD6E054F7F0E04404F02200020EB300020FC0
:400F06000400020E8900020F0FC0E0C083C082C085C084C086758600D2185391EF907FAB7408F0D086D084D085D082D083D0E0327400F58690FDA57C05A3E582458370F9B9
:400F460022907FD6E04480F04387010000000000220000000000000000000000000012011001FF000040CD0607010100010200020902430001010080320904000007FF008A
:400F86000000070501024000000705020240000007050302400000070581024000010705820240000107058302400001070584024000010403090410034B00650079007332
:170FC60000700061006E000E03530065007200690061006C00000064
:00000001FF
